S31508001800E0080020D9180008E7180008E9180008B9
S3150800181000000000000000000000000000000000BA
S315080018200000000000000000000000000119000888
S31508001830000000000000000003190008C93600086F
S31508001840B53F000807190008071900080719000816
S3150800185007190008071900080719000807190008DA
S315080018600719000899280008071900080719000829
S3150800187007190008071900080719000807190008BA
S3150800188007190008000000000000000007190008FA
S3150800189000000000071900080719000807190008C2
S315080018A00000000007190008071900080D3B00088A
S315080018B007190008071900080719000800000000A2
S315080018C0EE11AA550348854600F030FC004800474B
S315080018D0FD500008E00800200B4880F308880B48F4
S315080018E080470B480047FEE704207146084202D0AD
S315080018F0EFF3098001E0EFF30880714603F082FAFE
S31508001900FEE7FEE7FEE7FEE7E00800205D37000891
S31508001910C518000830B50B460146002020220124D0
S3150800192009E00D46D5409D4205D31D469540491B05
S315080019302546954040191546521E002DF1DC30BD4E
S3150800194070B500242546002801DA01244042002902
S3150800195001DA01254942FFF7DDFFAC4200D04042DB
S31508001960002C00D0494270BD03460B439B0703D0A9
S3150800197009E008C9121F08C0042AFAD203E00B7846
S315080019800370401C491C521EF9D27047D2B201E0BE
S315080019900270401C491EFBD270470022F6E710B5BC
S315080019A013460A4604461946FFF7F0FF204610BDBF
S315080019B0F8B502464A40D40F42004B0052085B086D
S315080019C09A4202D20246084611464A0023D0C30D5F
S315080019D04A00DDB2120EAD1A202D35DA490201266B
S315080019E0490AF6058A19002C00D0524220214F1BBD
S315080019F01146B9402A411018C20D9A4221D0002C2E
S31508001A0017D0012D08DCDA05801AD20F8019D20703
S31508001A10DBB200F0F2FAF8BDDA05801A01234000BD
S31508001A201B06C01880185A428018CA0F104349006E
S31508001A3007E04908C2071143DA05801A80194008E9
S31508001A40801800F0D2FAF8BD61000122511A001B75
S31508001A50F7E70122D2075140AAE70122D2075040F0
S31508001A60A6E7024670B54A40D30FDB0740002DD0E3
S31508001A704A002AD0010E140E000212020919400A61
S31508001A80520A8418E50104465443000A120A2E0431
S31508001A905043A4194219200CC543AA18120C012553
S31508001AA0AD03521C521912047F39240400D0521C6B
S31508001AB0104301D44000491EC2B20C06C0092018C2
S31508001AC0401C4008802A02D003E0002070BD400870
S31508001AD04000002900DA0020184370BD70B50246A0
S31508001AE04A40D50F40004A00ED0740085208002832
S31508001AF014D0002A12D0C40DD30D41020120C0050E
S31508001B005202490A520AE41A091812187D349142F7
S31508001B1001D3641C00E04900002C01DA002070BDE6
S31508001B200023914201D3891A03434008490000283B
S31508001B30F7D100290AD0914202D10121C90705E04F
S31508001B40914201D2012101E00121C943E005C018F3
S31508001B50401900F04AFA70BDF0B5074608465840E5
S31508001B6087B0C00F049048000E465900400849083F
S31508001B70BC1A884105D2384631461E4617460B46DA
S31508001B8002465800400810434CD0300D03904005DB
S31508001B905900400D490D0590401A0290402872DA06
S31508001BA018030121000B09050843019004980092C7
S31508001BB0002805D0019952420020884100920190E0
S31508001BC0029840210A1A0199009800F0EBF9054697
S31508001BD00C466B4607CB00F0F5F9C0197141039A1C
S31508001BE00E0D0023D71756401A467A40164344D09E
S31508001BF0049A002A2DD0029A012A039A15DC1205A6
S31508001C00C01A914101263605001C7141D20F059E66
S31508001C10D2070093019202962A46234600F033FA29
S31508001C2007B0F0BD38463146FAE71605224A0F4690
S31508001C30B218C01AB74101210905001C4F41001806
S31508001C407F41114618187941E20F10436D19644116
S31508001C5013E0E2076D0815436408C2071443039AA4
S31508001C6001261205C01A91413605001C7141CE079E
S31508001C70400830434908C01851412A46234600F017
S31508001C80F5F9CDE7FFE7049801224000C117121ABB
S31508001C9000238B4104983146C417381AA141EEE750
S31508001CA030B40124E407634030BC55E730B401245E
S31508001CB0E407614030BC4FE70000E0FFF0B51FB411
S31508001CC088B00B990998002448400999C00F490023
S31508001CD049080991C0070B990090490049080B91DA
S31508001CE009990898A64608431CD00B990A980843F0
S31508001CF018D0099801244000420D4800410D099862
S31508001D0024050003000B204309900B980003000BE1
S31508001D1020430B9050181C49401800220190144685
S31508001D20104605E0002001460DB0F0BD032801DA93
S31508001D30034600E003239C46C11A0AAE0AE05F0088
S31508001D4008ADED5B4F00F75B7D430027AA187C4181
S31508001D50491C5B1E6145F2DD410004AB5A52210461
S31508001D60120C0A43240C401C0828DFDB0198029059
S31508001D700099704601910090059B049A0799069868
S31508001D8000F081F9D0E700000DFCFFFFF0B50C4626
S31508001D905C4085B0E40FE40703944C000026640811
S31508001DA059009446490802460296224321D06246C3
S31508001DB00A431ED06200570D4A000E032303550D31
S31508001DC0012402462C492405781B1B0B360B4018A8
S31508001DD023432643614600901C46501AB44103D358
S31508001DE00098401C009002E0921800985B41002879
S31508001DF003DA0020014605B0F0BD002001210905DF
S31508001E000746864611E064461D46141BB54106D3AF
S31508001E106546521BB341744607430C43A646CD0795
S31508001E2040084908284392185B4105460D43EAD104
S31508001E301046184313D0604619465040714008436F
S31508001E4006D06046101AB34106D20122002306E0E6
S31508001E5000220123DB0702E00122D2435310009837
S31508001E6074460105381C6141029C039D00196941AD
S31508001E7000F0FCF8BFE70000FD030000C217C10F21
S31508001E80504010B54018CA079623002100F0B5F84F
S31508001E9010BD10B500229623114600F0AEF810BD0D
S31508001EA00EB505490291002100910A460B4601919B
S31508001EB000F0E9F803B000BD330400004100400219
S31508001EC00122400AD205090E80187F2901DA00206E
S31508001ED07047962903DC9622511AC84070479639EE
S31508001EE088407047C20FD207400040080BD0C10D8A
S31508001EF00723DB01C91840020905400A1143C20835
S31508001F00400711437047002001467047CB0FDB0797
S31508001F10490010B5490802460A4307D00A0D0724A6
S31508001F200903E401090B121B002A01DC002010BD7D
S31508001F30C900440F0C43C100E018D205801800F010
S31508001F4054F810BDF0B51FB40646002082B0054609
S31508001F504024019100901BE0019922460F46304625
S31508001F6000F0F6F8049A059B801A994110D310469A
S31508001F701946224600F016F8361A8F41019722466E
S31508001F8001200021009F00F00DF838184D410090FF
S31508001F902046641E0028DFDC019B0098294632464D
S31508001FA007B0F0BD10B5202A04DB0146203A91405F
S31508001FB0002010BD914020239C1A0346E340194394
S31508001FC0904010BD10B5202A06DBCB170846203AEC
S31508001FD01041C1170B4306E00B461341D04020249D
S31508001FE0A21A91400843194610BD002904DA401C7C
S31508001FF0490001D140084000704770B40024050C20
S3150800200005D11024000402D1002921D01124050E7F
S3150800201001D100020834050F01D10001241D850FE6
S3150800202001D18000A41C002801DB4000641C0029A3
S3150800203008D020252E1B0D46F540A14000D00121D1
S315080020402943084301061B1B000ADB1D02D5002095
S3150800205070BC7047DB05181880180029F8DA401C90
S315080020604900F5D170BC40084000704710B5002BF8
S3150800207008DA0024401C614192185B411A4301D1D9
S315080020804008400010BDF0B51FB482B005460C00EC
S3150800209003D0084601F0DCFF02E001F0D9FF20304A
S315080020A00246009021462846FFF77CFF049B059AC6
S315080020B004460F4618431143084314D018461043E4
S315080020C01BD0009840210A1A1846059900F040F8D6
S315080020D005460E46009A05990498FFF763FF0843DC
S315080020E005D0012004E02046394607B0F0BD00209F
S315080020F0C11705430E432C43374300990E986305D1
S31508002100401A7905E40A00220C43FD0A0A3002D572
S3150800211000200146E9E70105101969410C9C0D9D4F
S3150800212000196941FFF7A2FFDFE70000064C012509
S31508002130064E05E0E36807CC2B430C3C9847103461
S31508002140B442F7D3FFF7C2FB885C0008A85C000816
S3150800215010B5202A04DB0846203AD040002110BDDD
S315080021600B46D340D0402024A21A91400843194672
S3150800217010BD000010B50446002C08D10121092025
S31508002180C00600F005FE002000F05AF94BE0012CCD
S3150800219005D102210920C00600F0FAFD43E0022C11
S315080021A005D104210920C00600F0F2FD3BE0032C0E
S315080021B005D108210920C00600F0EAFD33E0042C09
S315080021C005D110210920C00600F0E2FD2BE0052C00
S315080021D005D120210920C00600F0DAFD23E0062CEF
S315080021E005D140210920C00600F0D2FD1BE0072CCE
S315080021F005D180210920C00600F0CAFD13E0082C8D
S3150800220004D101210A4800F0C3FD0CE0092C04D1D1
S315080022100221074800F0BCFD05E00B2C03D1102174
S31508002220034800F0B5FD204600F00AF910BD00008D
S3150800223000040048FEB5002000900190029000249A
S31508002240A3E000250DE006206843654940186100B3
S31508002250405AA1006A4651584018A1005050681CBF
S3150800226085B2142DEFDBA1006A4650581421FFF7FA
S3150800227051FB2821484361005A4A515A3C2251438E
S31508002280461864213046FFF745FB6100554A50520F
S3150800229055480079002806D160001146085AA10061
S315080022A0524A50506EE0012C01D0022C6AD14E4899
S315080022B02038407E002808D1012C06D16000494903
S315080022C0085AA100494A50505DE0A00047490858FD
S315080022D06100444A515A88422AD260001146085A77
S315080022E0A100424A5158401A0A2817D94048015DA8
S315080022F0005D401C3E4A1055142908DD0020114691
S31508002300085560003749085AA100384A5050A000BD
S315080023103649085A6100334A505233E0002034499E
S31508002320085560002F49085AA100304A505029E044
S31508002330A0002E49085861002A4A515A401A0A280C
S3150800234017D92B48015D005D401C294A10551429F0
S3150800235008DD00201146085560002249085AA100E8
S31508002360224A5050A0002149085A61001D4A50527D
S3150800237008E000201E49085560001A49085AA100BD
S315080023801A4A505000BF601C84B2032C00DA58E782
S3150800239015480079002822D01248408815498842F5
S315080023A003DC10488088884208DD0F482038407DC5
S315080023B0002803D101210C48203841750948408876
S315080023C00A2803DB074880880A2808DA06482038DE
S315080023D0407D002803D10121034820384175FEBD00
S315080023E05403002014010020D4020020CC0300204E
S315080023F021010020E60F000000B587B001A800F013
S31508002400AFF80121480200F0D1FF002001907020AA
S31508002410029001208002039000200690059001A9F1
S31508002420064800F031F80121044800F021F801219E
S31508002430024800F011F807B000BD00000024014072
S3150800244010B50446072300222146024800F038F852
S3150800245010BD000000240140002904D04268012371
S315080024601A43426003E042685208520042607047CD
S31508002470002904D0826808231A43826003E0826830
S3150800248008239A438260704742680B4B1A404260A1
S315080024900B684A681A4343681A4342608268074BC6
S315080024A01A4082600B694A691A438B681A43836823
S315080024B01A438260704700000FBCFFFF8FF1F9FFD7
S315080024C0F0B504460D4616461F463F073F0F2B46F6
S315080024D0082B0FD91B071B0F083B606F9A000F21AB
S315080024E0914088436067606F99003A468A40104376
S315080024F060670BE0206F9A000F21914088432067A0
S31508002500206F99003A468A4010432067E068012107
S31508002510A9408843E060E0680121A9400843E060DB
S31508002520012080032840002803D0012000F020F86D
S3150800253007E00120C0032840002802D0012000F04F
S3150800254017F8F0BD002905D08268FF2301331A4326
S31508002550826004E08268FF2301339A4382607047F1
S31508002560002101604160816001730161416170472A
S31508002570002806D0064949680C221143044A5160CE
S3150800258005E0034949680C229143014A51607047A6
S315080025900024014010B523480078012835D10020D1
S315080025A0204908702049088013E01F480088400029
S315080025B01E49095A1E480088062250431D4A80189B
S315080025C0194A12885200815217480088401C164939
S315080025D00880154800880328E7DB7E2001F0F6FC12
S315080025E0022000F02BF901211348FFF7ABFF104832
S315080025F00088401C0E49088008460088142804DB19
S315080026000020088001200D4908700C480078002831
S3150800261006D0FFF70FFE00200849087000F002FCFC
S3150800262010BD0000200100203A01002020030020F0
S315080026303C01002054030020002401401A01002018
S31508002640FFB583B00C46029400200190002726E0CF
S3150800265000261CE0721C039951430846791CFFF7B3
S3150800266059F90546A54201D9281B00E0601B054615
S315080026700298A84204D9029505980670069807702C
S315080026800298002802D10120019002E0761C402E13
S31508002690E0D300BF0198002800D002E07F1C042F79
S315080026A0D6D300BF029807B0F0BD000000BF00BF38
S315080026B000BF00BF00BFBFF34F8F00BF00BF00BF02
S315080026C006480749C86000BF00BF00BFBFF34F8F69
S315080026D000BF00BF00BF00BF00BFFDE70400FA054A
S315080026E000ED00E010B500F001F810BD10B5234864
S315080026F00078002817D1224800F0E0FE01283CD1D6
S315080027001F480078002838DD1D480078402834DC4A
S3150800271001F0CFF91B49086001201849087000200C
S315080027201949087029E0164A17490978491C5018AA
S3150800273000F0C4FE012816D113480078401C12493F
S3150800274008700F4800780978884216D100200B498E
S3150800275008700B484078FF280FD10B4800780228EC
S315080027600BD1FFF7A3FF01F0A4F906490968643104
S31508002770884202D900200149087010BDED000020EA
S31508002780DC020020F0000020EC00002010B586B026
S3150800279004460121880300F009FE0121480400F0DF
S315080027A0E5FD01220921C80600F0DDFA01220A2109
S315080027B00920C00600F0D7FA01A801F080FA0194B2
S315080027C030216846018100214181818101821821D9
S315080027D0C18101A9184801F02FFA0121164801F014
S315080027E008FA05A800F015FB01214902684681820E
S315080027F0012181751821C17505A90920C00600F0B7
S3150800280065FA01218902684681824821C17505A9B0
S315080028100920C00600F05AFA1B21684601700321F8
S3150800282041700121817000F06DFD012202210248EC
S3150800283001F0F7F906B010BD0038014001B50449AA
S315080028400098086000BF024800680028FBD108BD50
S31508002850F4000020014600220E4B1A61CA005A6194
S3150800286000229A6105221A6100BF0A4A1069C20746
S31508002870D20F002A04D0012212040240002AF4D002
S31508002880044A126952085200024B1A6100229A61E0
S315080028907047000000E000E010B500210448FFF78B
S315080028A051FE022000F04AF801200249087010BDC6
S315080028B0002401402001002000B589B00121084606
S315080028C000F054FD1A4800F045F801A800F08EF80B
S315080028D018480190184802900021684601730320A1
S315080028E0049068460175802141754900C1828900B6
S315080028F0018320218176090281830021C183018415
S3150800290001A90B4800F04CF80121094800F01CF811
S3150800291001220221064800F039F8092168460170AB
S31508002920022141700121817000F0ECFC09B000BD64
S3150800293008000240002401402003002001494860A5
S3150800294070470000000002400268520852000A431D
S315080029500260704710B504462068400840002060B1
S31508002960002020606060A060E060E1B20846083898
S315080029700521FEF7CFFF01460F2088400249496826
S3150800298008430149486010BD00000240002A03D0F0
S3150800299003680B43036002E003688B4303607047D8
S315080029A010B50A7A8B7D1A430B7C1A434B7C1A4363
S315080029B04B8A1A438B8A1A430B8B1A434B8B1A433F
S315080029C00368094C23401A43026002680123DB03AB
S315080029D09A438B8B1A430260CA6842600A6882600F
S315080029E04A68C26010BD00000F80FFFF0021016029
S315080029F041600172C16001744174418281828175AE
S31508002A00018341838183704770B506460C4621468B
S31508002A100A4800F0FBF80546002D01D1401E70BD9E
S31508002A200648854202D10648051B00E02D1B2246B2
S31508002A3029463046FEF798FF2046F0E700F40008DE
S31508002A4000FC000870B505460C4622460249284691
S31508002A5000F09DF8204670BD00F4000810B5044645
S31508002A600848006902210843064908610846446186
S31508002A7000694021084303490861034800F006F944
S31508002A8010BD000000200240FF0F00000C48C0687F
S31508002A90C007C00F002801D0012070470848C06849
S31508002AA004210840002801D00220F6E70448C0683F
S31508002AB010210840002801D00320EEE70420ECE7A7
S31508002AC00020024003480069802108430149086143
S31508002AD0704700000020024030B504460D46054800
S31508002AE00069012108430349086125800F2000F089
S31508002AF0CDF830BD0020024010B57E2001F066FA00
S31508002B00034800F007F87E2001F060FA10BD0000C7
S31508002B1000F4000810B5044600F0ACF82046FFF7AC
S31508002B209DFFFFF7CFFF10BD70B5034601250022B4
S31508002B3008E050001C5A0748844201D0002506E0E8
S31508002B40501C82B2CE0F761876109642F1DC00BF82
S31508002B50284670BDFFFF0000F8B505460E46144628
S31508002B6000F088F87E2001F031FA002707E029886E
S31508002B703046FFF7B1FFB61CAD1C781C87B2E10FD3
S31508002B8009194910B942F2DCFFF79CFFF8BDF8B500
S31508002B9007460C4615462946204600F037F80646ED
S31508002BA0002E0DD12046FFF7B5FF01208002201820
S31508002BB0FFF7B0FF2A4621463846FFF7CDFF24E047
S31508002BC0012080022018401BB0420AD10120800251
S31508002BD02018FFF79FFF2A4631463846FFF7BCFF05
S31508002BE013E00120C0022018401BB04208D120463D
S31508002BF0FFF790FF2A4631463846FFF7ADFF04E057
S31508002C002A4631463846FFF7A7FFF8BDF8B5054608
S31508002C100E462F46E807C00F002801D000BFFEE782
S31508002C2031460120C002FEF78BFE002901D000BF05
S31508002C30FEE700240BE02046704347193146384624
S31508002C40FFF772FF012800D108E0601C84B2314604
S31508002C500120C002FEF774FEA042ECDC00BF31463C
S31508002C600120C002FEF76CFEA04200D100273846BC
S31508002C70F8BD0000024803494860034848607047A9
S31508002C802301674500200240AB89EFCD10B5024607
S31508002C9000BFFFF7FBFE0346521EFF2400E0641E3A
S31508002CA0002CFCD1012B01D1002AF2D1064800697B
S31508002CB077218843044908613420C860002A01D175
S31508002CC0052010BD1846FCE700200240F8B502466C
S31508002CD0CD782F073F0FCD7810263540002D01D02F
S31508002CE08D782F431446002011E085062B0E0D889B
S31508002CF0012686403540002D07D025680F269E40C0
S31508002D00B5433E469E4035432560451CE8B2082833
S31508002D10EBDB141D0D882D120095002011E08506A9
S31508002D202B0E01258540009E3540002D07D02568CD
S31508002D300F269E40B5433E469E4035432560451CBA
S31508002D40E8B20828EBDBCD78282D04D155690E8822
S31508002D503543556106E0CD78482D03D115690E88AF
S31508002D6035431561F8BD70B54D07EB0E082902DA33
S31508002D700546203501E0054624352C460F269E409B
S31508002D802568B54316469E403543256070BD00004C
S31508002D9038B504460D460920C006844203D10121F0
S31508002DA0480400F0E3FA1148844203D101210002E5
S31508002DB000F0DCFA0E48844203D10121000200F03B
S31508002DC0D5FA0C48844203D10121080500F0CEFA51
S31508002DD0684600F01EF868460580012181700021CA
S31508002DE0C17069462046FFF771FF38BD00040048E8
S31508002DF000080048000C0048024690680840002871
S31508002E0001D0012070470020FCE74161704701614D
S31508002E1070470021C9430180022181700421C170D5
S31508002E2070470000F0B58FB00025002600200D90F1
S31508002E300C907E2001F0CAF800241AE06100B34A1B
S31508002E40505AFFF726F8B2490790FEF747FE07469D
S31508002E50FFF748F80022AF4B09910890FEF72EFFBE
S31508002E600B910A90FFF752F8A100AB4A5050601C2C
S31508002E7084B2032CE2DBA8498868FFF733F8A74A2F
S31508002E80A74B05910490FEF70BFF0022A54B07916F
S31508002E900690FEF77BFFA44AA44B09910890FEF71B
S31508002EA005FF0B910A90FFF731F805469A494868DD
S31508002EB0FFF718F89E4A9F4B05910490FEF7F0FE1F
S31508002EC00022984B07910690FEF760FF964A974BAB
S31508002ED009910890FEF7EAFE0B910A90FFF716F89B
S31508002EE006462846FEF7FEFF00228A4B0591049007
S31508002EF0FEF7DCFE0991089029468F48FEF7B1FDDA
S31508002F000746FEF7EFFF07910690099B089AFEF71A
S31508002F103DFF0B910A90FEF7F9FF88490860304695
S31508002F20FEF7E0FF00227B4B05910490FEF7BEFEFC
S31508002F300991089031468048FEF793FD0746FEF74B
S31508002F40D1FF07910690099B089AFEF71FFF0B9180
S31508002F500A90FEF7DBFF7A4908607A49088BFEF784
S31508002F609FFF794A794B03910290FEF7A7FE00224C
S31508002F70774B05910490FEF709FF0991089071496E
S31508002F80088BFEF786FF0746FEF7ACFF0022704B5C
S31508002F9001910090FEF7FAFE0591049067480068D3
S31508002FA0FEF7A0FF03910290059B049AFEF778FEB0
S31508002FB007910690099B089AFEF7E8FE0B910A907E
S31508002FC0FEF7A4FF0D905F49488BFEF769FF5E4A3E
S31508002FD05E4B03910290FEF771FE00225C4B059151
S31508002FE00490FEF7D3FE099108905649488BFEF7E0
S31508002FF050FF0746FEF776FF0022554B01910090D9
S31508003000FEF7C4FE059104904D480068FEF76AFF76
S3150800301003910290059B049AFEF742FE07910690DB
S31508003020099B089AFEF7B2FE0B910A90FEF76EFF0F
S315080030300C9048480D99FEF7BBFC0746FEF73EFF85
S315080030404549086043480C99FEF7B2FC0746FEF767
S3150800305035FF424908603B48D830008D3E4909682B
S315080030604018C003010C3748D8300185408D3B49CC
S3150800307009684018C003010C3248D83041852649F2
S3150800308008683749FEF7EDFC0746FEF717FF81B2D9
S315080030902C48D83081852030C07D00282AD129487F
S315080030A0D830808DFD2804DC00212648F83081734D
S315080030B00FE02448D830808DFF211731884204DC80
S315080030C001212048F830817303E002211D48F830B9
S315080030D081731C48F830017E007E401CC2B2194834
S315080030E0F83002760F2901DD0121C1750020154946
S315080030F028394860134828380088642803DD0020EA
S315080031001049283908800FB0F0BD000014010020CE
S3150800311000F07F4500000840480300209A999999D5
S315080031209999C93F0000284025068195438BD43FCD
S31508003130333333333333C33F000048432801002079
S315080031402C010020BC010020091B9E5E29CB703F84
S3150800315000408F400000C8413001002034010020A3
S315080031600000C8420148006870470000F8000020C7
S315080031700348006803490978401801490860704700
S31508003180F80000200001002008B50121480400F0DD
S31508003190EDF80121880400F0E9F86846FFF739FEE2
S315080031A00121C903684601804821C1706946092082
S315080031B0C006FFF78BFD6846FFF72BFE01210903C2
S315080031C0684601804821C17069460920C006FFF794
S315080031D07DFD6846FFF71DFE4021684601800421F3
S315080031E0C17069460148FFF771FD08BD0004004833
S315080031F010B50121C9030920C006FFF7FDFD002807
S3150800320008D12148807E002808D101211E488176F0
S31508003210C17403E000211C48C17481761B4880688C
S315080032207D21090188422CD900201849886000218F
S315080032301548C1742030007900281CD1082114488B
S31508003240FFF7E5FD1048807B00280CDD0E48203886
S31508003250408D822804DA01210B482030017102E0F2
S315080032600121094841750848807C012809D10020B8
S315080032700649486005E000200449486000210248E4
S3150800328081740148C07C10BDB4020020940100205E
S315080032900004004808B50121480400F067F8012138
S315080032A0880400F063F86846FFF7B3FD0D21684609
S315080032B00180012181701021C17069461048FFF70D
S315080032C005FD8E2168460180012181701021C1709B
S315080032D069460920C006FFF7F9FC08210920C0063F
S315080032E0FFF793FD80210920C006FFF78EFD012117
S315080032F00348FFF78AFD08210148FFF788FD08BD46
S31508003300000400488178002925D0174903221202B3
S315080033108918027892109200895802789207D30E7B
S31508003320FF229A40914342789207120E03789B0730
S31508003330DB0E9A4011430C4A03231B02D21803786A
S315080033409B109B00D1500178CA06D20E01219140EC
S31508003350054A116007E00178CA06D20E012191409C
S31508003360014A80321160704700E100E0002905D06B
S31508003370054A52690243044B5A6104E0024A5269FB
S315080033808243014B5A61704700100240002905D05C
S31508003390054AD2690243044BDA6104E0024AD2695B
S315080033A08243014BDA61704700100240002905D0BC
S315080033B0054A92690243044B9A6104E0024A9269FB
S315080033C08243014B9A6170470010024010B500F025
S315080033D031F804494968F02211400909024A515C4A
S315080033E0C84010BD00100240C800002010B5FFF705
S315080033F0EDFF05494968072212021140090A034AE6
S31508003400515CC84010BD000000100240C8000020F2
S3150800341010B5FFF7DBFF054949680722D2021140BC
S31508003420C90A034A515CC84010BD0000001002409A
S31508003430C8000020F8B51E4840680C21084004283A
S3150800344002D008282ED101E01A4C2DE01848403049
S315080034500069C007C00F00280AD015484030006927
S3150800346002210840002801D0134802E0114800E074
S31508003470104807460E4840300069FF2109040840F5
S31508003480000C451C0A48403000690721090208401B
S31508003490000A461C3946694308463146FEF73AFA99
S315080034A0044601E0034C00BF00BF2046F8BD0000FB
S315080034B00010024000127A0000093D0070B504466B
S315080034C000250221074800F09AFB002808D0054885
S315080034D000F0EEFB20700221024800F088FB01256F
S315080034E0284670BD0038014010B500F001F810BD3F
S315080034F000B585B062480068012108436049086044
S3150800350000BF5F480068022108400028F9D05D48DE
S315080035105D4908605D480068102108435B490860FA
S3150800352008460068C008C000086057490968481E70
S315080035305749FEF7EFF9049054480068049949077B
S31508003540490F0843514908604D48406851490840A9
S315080035504B494860084640689021084348494860F6
S31508003560084640684860484800684649884207D97E
S3150800357043484068052109020843414948600BE071
S31508003580414800684449884206D93D4840680121B7
S31508003590890208433A4948606B4601AA3A480168D5
S315080035A03E48FFF74DF836484030006980088000ED
S315080035B033494031086108460069400840000861FF
S315080035C0684600784007400F029068460079400632
S315080035D0400E03902A48C069890508432849C861EE
S315080035E02748403000692E4908402549403108617E
S315080035F003980004029909020843214940310969E0
S3150800360008431F49403108611D4800680121090621
S3150800361008431B49086000E000BF194800680121FB
S31508003620490608400028F7D01548406880088000F9
S315080036301349486008464068022108431049486013
S3150800364000E000BF0E4840680C2108400828F8D161
S315080036500120FFF7FFF80A48406810218843084907
S3150800366048600120FFF7F6F805484068802188433E
S31508003670034948600120FFF7EDF805B000BD0000DA
S315080036800010024000A24A04D80000200020024090
S3150800369000366E010FC0FFFF0051250200127A00A6
S315080036A0FFF800FF042806D10649096904221143D8
S315080036B0044A116105E00349096904229143014A54
S315080036C01161704700E000E010B5FFF751FD204892
S315080036D00088401C1E49088008464068401C48600F
S315080036E01C480068002804D01A480068401E19497A
S315080036F008601948C07C01280CD117482030007989
S31508003700002801D11249486011488068401C1049B8
S31508003710886002E000200E4988600F48007C012876
S3150800372005D10B480069401C0949086102E00020E0
S31508003730074908610848807D012805D10448006AC0
S31508003740401C0349086202E000200149086210BDD6
S3150800375094010020F4000020B402002010B5164899
S31508003760006801210843144908600846406813495F
S3150800377008401149486008460068114908400E4942
S315080037800860084600680121890488430A490860D8
S3150800379008464068C3210904884307494860084623
S315080037A0006808490840044908609F2000048860AA
S315080037B0FFF79AFE10BD0000001002400CC0FFF88B
S315080037C0FFFFF6FEFFFF8F0008B501214804FFF74B
S315080037D0CDFD022201210920C006FFF7C4FA022105
S315080037E0684601801821C170012181706946092047
S315080037F0C006FFF76BFA01214804FFF7B7FD02225E
S3150800380011460920C006FFF7AEFA04216846018072
S315080038101821C1700121817069460920C006FFF789
S3150800382055FA08BD30B587B004460D46012108464D
S31508003830FFF7ACFD04A800F033F905946846058245
S31508003840002101838176817404A90120800700F094
S31508003850F1F8684600F0D2F8602168460170012147
S3150800386041700020019000216846017269460120D6
S31508003870800700F057F869460120800700F08AF8AB
S315080038800821C80600F07EF80821C80600F0B0F83E
S315080038904021080600F038F84021080600F03CF8F8
S315080038A00121880700F00AF80121880700F01EF8B0
S315080038B00121880700F00EF807B030BD002904D0B2
S315080038C0026880231A43026003E0026880239A4351
S315080038D002607047002904D0026801231A43026077
S315080038E003E002685208520002607047002905D0BA
S315080038F0426C0123DB031A43426404E0426C012351
S31508003900DB039A4342647047826907231B039A4381
S315080039100B021A4382617047C26970239A430A43AD
S31508003920C261704710B5826907231B039A430B7857
S315080039301B021A4382610A7A12014B781B011A4349
S31508003940036A3024A3431A4302624A6882630C4A14
S31508003950904213D14A7A12018B781B011A43036AE3
S31508003960C024A3431A4302624A8992008B899B00AA
S315080039701A4343682401A3431A43426010BD00005A
S31508003980002C014082690123DB029A430B021A4389
S315080039908261704710B5C26970239A430B781A433F
S315080039A0C2610A7A12024B781B021A43036A03247D
S315080039B02402A3431A4302624A68C2630B4A90422E
S315080039C013D14A7A12028B781B021A43036AA4009F
S315080039D0A3431A4302624A8912018B891B011A43BF
S315080039E04368A400A3431A43426010BD002C01405B
S315080039F0C26908239A430A43C261704700210170CD
S31508003A0041708170416001724172418181817047C4
S31508003A1001229207904201D1816301E08AB2826352
S31508003A20704701229207904201D1C16301E08AB230
S31508003A30C2637047026803231B029A430B891A4321
S31508003A400260134A904206D001229207904202D0A1
S31508003A50104A904205D1026870239A438B781A431C
S31508003A6002600B4A904205D00B4A904202D00B4A9C
S31508003A70904205D1026B120A12028B7A1A4302632C
S31508003A804A68C2620A88826201224261704700005F
S31508003A90002C014000040040004401400048014059
S31508003AA00021C94341600021018001818170817232
S31508003AB0704710B5FFF756FB10BD000070B5FFF74D
S31508003AC085FC05467D21C900FDF724FF0446601ED6
S31508003AD00C49884200D90CE0601E0B494861032155
S31508003AE0081F00F0DBFA00200749886107200861F3
S31508003AF000BF0420FFF7D6FD0021481E00F0CEFACD
S31508003B0070BD0000FFFFFF0000E000E010B50221D5
S31508003B10154800F07DF8002824D0134800F0C8F8AE
S31508003B20C4B21248007C002803D1204601F022F8CE
S31508003B3014E00E48007C022810D10C48407C00286E
S31508003B400CD10B488079AA2804D10948C4710121EF
S31508003B5006484174AA2C01D10548847102210248FD
S31508003B6000F045F810BD000000380140B4020020FE
S31508003B70D803002010B504462146054800F09CF8F5
S31508003B8000BF0121024800F03AF80028F9D010BD1C
S31508003B900038014070B505460E4600247E2000F028
S31508003BA015FA00BF20E0042C19DD701EA04216DDB0
S31508003BB0285D7E2806D17D20FFF7DCFF5E20FFF713
S31508003BC0D9FF0FE0285D7D2805D1FFF7D3FF5D20DB
S31508003BD0FFF7D0FF06E0285DFFF7CCFF02E0285D7F
S31508003BE0FFF7C8FF601C84B2B442DCDB70BD4161DC
S31508003BF070478269520852000A438261704702463A
S31508003C0090680840002801D0012070470020FCE792
S31508003C100246D0680840002801D0012070470020DD
S31508003C20FCE7002A03D003690B43036102E003693A
S31508003C308B4303617047000070B504460D460026A5
S31508003C40E0693021884329790843E061E069442125
S31508003C508843A9790843E061E06980088000297AE9
S31508003C600843E061A0691821884369890843A0616F
S31508003C70A06904218843297B0843A0610B48844234
S31508003C8003D1FFF7C5FB064602E0FFF7AFFB064682
S31508003C9030462968FDF73EFE00092062304629684D
S31508003CA0FDF738FE0007000F606270BD003801405E
S31508003CB001464868C0B27047CAB2026070474B21D5
S31508003CC0C901016030210171002181710172182139
S31508003CD0418100210173704710B5A548807B030018
S31508003CE000F0CDF905045A93DAFBFA00A04820380B
S31508003CF0808DFD280DDB9E48F838808B012805D17C
S31508003D0000219B48F838818300F006FF0121984876
S31508003D10817340219748FFF76FF8002815D0964918
S31508003D204868FF21F531FDF7F5FDC007C00F0028EB
S31508003D3005D180210920C006FFF767F822E0802117
S31508003D400920C006FFF763F81CE08B494868C821BC
S31508003D50FDF7E0FDC007C00F002805D18021092026
S31508003D60C006FFF752F80DE083494868C821FDF7F9
S31508003D70D1FDC007C00F002804D080210920C00645
S31508003D80FFF745F808210920C006FFF73EF801218C
S31508003D907848FFF73AF8E8E075482038808DFF2123
S31508003DA01731884202DB022171488173402171482C
S31508003DB0FFF722F8002813D06F494868FF21F5312C
S31508003DC0FDF7A8FDC007C00F002804D101216948E6
S31508003DD0FFF71BF80EE001216648FFF718F809E01F
S31508003DE065484068FF21F531884203D901216148B9
S31508003DF0FFF70DF880210920C006FFF706F808210D
S31508003E000920C006FFF701F8AFE059482038808D31
S31508003E10FF212531884202DD03215548817340215F
S31508003E205448FEF7E9FF002827D053494868FF2180
S31508003E30F531FDF76FFDC007C00F00280ED18021B0
S31508003E400920C006FEF7E3FF01214A48FEF7DFFF17
S31508003E5008210920C006FEF7DAFF1CE080210920A8
S31508003E60C006FEF7D2FF08210920C006FEF7CDFFDF
S31508003E7001214048FEF7C9FF0DE080210920C00650
S31508003E80FEF7C5FF01213B48FEF7C1FF08210920BF
S31508003E90C006FEF7BCFF68E040213648FEF7ACFFD7
S31508003EA0002843D0012109030920C006FEF7A4FF14
S31508003EB0002813D180210920C006FEF7A8FF01219A
S31508003EC02C48FEF7A4FF08210920C006FEF79FFF2D
S31508003ED004212748817337E046E036E026494868DA
S31508003EE0FF21F531FDF716FDC007C00F00280ED1DA
S31508003EF080210920C006FEF78AFF01211D48FEF72A
S31508003F0086FF08210920C006FEF781FF1CE08021F4
S31508003F100920C006FEF779FF08210920C006FEF72A
S31508003F2074FF01211348FEF770FF0DE08021092078
S31508003F30C006FEF76CFF01210E48FEF768FF082150
S31508003F400920C006FEF763FF0FE080210920C0069E
S31508003F50FEF75DFF01210748FEF759FF08210920F2
S31508003F60C006FEF754FF00E000BF00BF10BD00000A
S31508003F70B402002000040048940100200348806829
S31508003F80400840000149886070470000002C004046
S31508003F9080210143014A116070470000002C00404F
S31508003FA003488068002801D0012070470020FCE7FC
S31508003FB0002C004010B5FFF7F3FF002804D0FFF7E8
S31508003FC0DDFF662000F002F810BD00004106490E2C
S31508003FD0014A116070470000002C004004494968F6
S31508003FE0FF22813291430143014A51607047000024
S31508003FF0002C004004494968C909C9014206520E05
S315080040001143014A51607047002C004070B50546BF
S315080040100C460121C802FFF7B9F9FF208130FFF7E6
S31508004020DDFF2046FFF7E6FF2846FFF7B1FF70BD24
S315080040300FB410B503A9044B044A029800F07AF8A5
S3150800404010BC08BC04B01847514B0008900100206A
S315080040502021020C01D010211046020A01D0104678
S315080040600839020901D01046091F820801D01046F6
S31508004070891E420801D0881E7047081A704730B456
S315080040807446641E2578641CAB4204D3635D5B00EA
S31508004090E31830BC18471D46F8E7000010B500289D
S315080040A019DB1A4A03231B02D21883089B00D2582D
S315080040B08307DC0EFF23A3409A438B071B0E840756
S315080040C0E40EA3401A43114B032424021B19840847
S315080040D0A4001A5118E00E4A03071B0F083B9B0859
S315080040E09B00D2588307DC0EFF23A3409A438B0715
S315080040F01B0E8407E40EA3401A43054B0407240F3E
S31508004100083CA408A4001A5110BD000000E100E014
S315080041101CED00E002E008C8121F08C1002AFAD107
S3150800412070477047002001E001C1121F002AFBD129
S3150800413070470000FFB58FB00F460446002606E01C
S3150800414025280AD0129A11999047641C761C207863
S315080041500028F5D1304613B0F0BD00250121A14A4B
S31508004160009500E00543641C23780846203B9840E8
S315080041701042F7D120782E2815D1042005436078FF
S31508004180641C2A280AD101CF641C00900BE0009910
S315080041900A22514330394018641C009020780146A1
S315080041A030390929F3D920786C280ED004DC4C283C
S315080041B013D06A2812D104E074280ED07A280DD1BB
S315080041C00BE001204005054307E001210905627857
S315080041D00D43824201D16D18641C641C2078864602
S315080041E069284AD008DC0028B4D058286DD063283E
S315080041F010D0642808D140E070286BD0732812D0FC
S31508004200752860D0782860D0129A70461199904720
S31508004210761CE5E03878694608720020487202A8DC
S315080042200190012003E0386801900020C0433F1D3B
S3150800423069070CD5002500E06D1C00998D420FDA40
S315080042408542F9DB0199495D0029F5D108E0002589
S3150800425000E06D1C8542FCDB0199495D0029F8D117
S31508004260761907E0019801990078491C0191129A7C
S31508004270119990476D1EF5D2B2E00A2002900021EE
S315080042806802400F039102280CD001CFC11784465B
S3150800429000290DDA624608465242002181419446B9
S315080042A02D2008E0FF1DFF08FF0003CF8446EFE737
S315080042B0280504D52B206A46107401203CE0E8073F
S315080042C03AD02020F7E70A2000E0102000210391C9
S315080042D0029007E0102002900021042005430820E0
S315080042E0039100906802400F022810D001CF0021E8
S315080042F0844600200D9028071FD5704670280CD0DC
S31508004300029A1020039B42401A430CD015E0FF1D69
S31508004310FF08FF0003CF8446EBE740206A46107487
S3150800432001200D900CE06046084306D030206A460E
S3150800433010747046507402200D907046582804D0A8
S3150800434029A001900DA80E900DE02CA0F9E7604673
S31508004350039B029AFDF7F6FD019B84469B5C0E9A29
S31508004360521E0E92137060460843F0D10E9805A9A6
S31508004370081A20300190680701D5009801E001204D
S3150800438000900199884203DD01460198081A00E069
S3150800439000200025009006E004A8129A405D1199B5
S315080043A090476D1C761C0D988542F5DB04E0129A41
S315080043B0302011999047761C0099481E00900029D4
S315080043C0F5DC08E00E980E990078491C0E91129AB1
S315080043D011999047761C0199481E01900029F1DC35
S315080043E0641CB4E6092801003031323334353637D7
S315080043F03839616263646566000000003031323323
S3150800440034353637383941424344454600000000C2
S3150800441010B502460023002901D1002010BD03E093
S315080044201488921CE01883B208464C1EA1B20028D4
S31508004430F6D11846F2E70000F8B500270026002452
S315080044400025F848407C01286FD17E20FFF7BEFD85
S31508004450F548C0790002F449097A08430746F24844
S31508004460467A847A0246D17A107B00F0BFFC05466C
S315080044700021EC484174ED49781A8F426FD01EDC52
S31508004480EB49781A8F426BD010DCEA49781A8F42CA
S3150800449067D006DC442F1CD0E7483818002872D1AC
S315080044A0DCE1882870D08928F9D16CE101286CD024
S315080044B002286BD003286AD00428F0D135E103001E
S315080044C0FFF7DDFD0C61C0FAF861611926768E41A9
S315080044D05C61062E09D1D948007800280AD100F077
S315080044E075FF0120D549087004E0152E02D1012078
S315080044F000F06CFFD0E1CB4820300079002806D0C8
S31508004500C8482038028D418D002000F0B9FEC3E16D
S31508004510002C0BD1C3482038408D00231A46F021C1
S315080045200090FE2000F0E1FE0CE0B6E1012C09D176
S31508004530BC482038008D01230022F0210090FE207F
S3150800454000F0D3FEA8E1002C0CD1BD48408D002315
S315080045501A46F3210090FE2000F0C7FE0DE05AE04F
S3150800456053E189E1012C08D1B548808E0123002248
S31508004570F3210090FE2000F0B8FE8DE1002C07D153
S31508004580AF48458506E086E111E11AE16AE07AE07E
S31508004590AB488586AA48808EFF21F531884206DA1F
S315080045A000F0BAFA0022FE21F42000F0D2FE73E1F0
S315080045B0002C09D1A248808D00231A46F1210090CB
S315080045C0FE2000F092FE0AE0012C08D19C48C08E1D
S315080045D001230022F1210090FE2000F086FE5BE117
S315080045E0002C02D19648858503E0012C01D1944818
S315080045F0C5869348808DFF21F53188420ADC9048AC
S31508004600C08E884206DC00F087FA0022FE21F220DE
S3150800461000F09FFE40E1002C09D18948C08D002397
S315080046201A46E9210090FE2000F05FFE09E0012C01
S3150800463007D1192001230022E9210090FE2000F06D
S3150800464054FE29E1002C01D17D48C585FF202D3077
S31508004650854206DA00F060FA0022FE21EA2000F020
S3150800466078FE19E1002C0CD17548008E6421484368
S3150800467080B200231A46E2210090FE2000F035FEA3
S3150800468000E000BF08E1002C06D164212846FDF7AA
S3150800469057F981B26A4801866948008EFF21F531CB
S315080046A0884206DC00F038FA0022FE21E32000F0FA
S315080046B050FEF1E01EE0FFE7002C0CD16048408E6A
S315080046C06421484380B200231A46EB210090FE205D
S315080046D000F00BFE0DE0012C0BD15948008F642128
S315080046E0484380B201230022EB210090FE2000F00F
S315080046F0FCFDD1E0002C07D164212846FDF720F9FE
S3150800470081B24F48418608E0012C06D1642128462B
S31508004710FDF716F981B24A48018700F0FDF9002233
S31508004720FE21EC2000F015FEB6E0012C13D13D4821
S31508004730807B002806DD01213A48203001710020DF
S315080047403F4948600022FE21E42000F002FE0121D4
S315080047503448817416E0002C0FD100213148817449
S31508004760203001710022FE21E42000F0F2FD002035
S31508004770324908703249486004E00022FE21E420EC
S3150800478000F0E7FD88E0002C0FD12748C07A3228D0
S315080047900CDC2548C17A2A48418700F0BDF9002279
S315080047A0FE21DF2000F0D5FD00E000BF74E02448BC
S315080047B0408F00231A46DE210090FE2000F095FD6A
S315080047C06AE0002C0FD11848C07A32281CDC16483B
S315080047D0C17A1B48818700F09FF90022FE21E1205B
S315080047E000F0B7FD10E0012C0ED10F48C07A322830
S315080047F00ADC0D48C17A1248C18700F08DF90022FB
S31508004800FE21E12000F0A5FD46E0002C1AD10C4857
S31508004810808F00231A46E0210090FE2000F065FDF7
S315080048201BE00000B4020020D8030020E9FE0000C7
S31508004830E0FE000056FE0000AB01FFFF8C010020E1
S3150800484094010020012C08D11448C08F01230022AE
S31508004850E0210090FE2000F048FD1DE0002C07D165
S3150800486001210F480174002202210E48FFF7D9F9E9
S315080048700DA0FFF7DDFB0FE0002C0BD1FF21013166
S315080048800A48FDF78AF800200849891F088002218E
S315080048900348017400E000BF00BFF8BD9401002082
S315080048A0B40200200038014031323300DE03002014
S315080048B0F0B589B000200890079006903D48407CE6
S315080048C0012874D13C488079AA286DD13A48C07924
S315080048D0322869DA3848C079002865DD3649C97949
S315080048E008461938FDF7CAFA08900898FDF7FAFA43
S315080048F00446324A324BFDF7E1F90022314B019169
S315080049000090FDF729F9039102902F480068FDF7FA
S31508004910E9FA0646039B029AFDF738FA05910490D0
S31508004920FDF7F4FA079029490798FDF79AF804461F
S31508004930FDF7C4FA81B21F48F83801830898FDF7D5
S31508004940D1FA06461D4A1E4BFDF7B8F90446002261
S315080049501C4BFDF701F9039102901D480068FDF70D
S31508004960C1FA01910090039B029AFDF70FFA05918F
S315080049700490FDF7CBFA069014490698FDF771F8EE
S315080049800446FDF79BFA81B20A48F838418300F0DD
S31508004990C3F80848F838428B018B0EA0FFF748FB8E
S315080049A0002104480174817400210248417409B049
S315080049B0F0BD0000B4020020D8030020091B9E5E4B
S315080049C029CB703F0000F03F2801002000007A4400
S315080049D02C010020525F30203A20202564202052E6
S315080049E05F313A2020202564200D0A0070B505465F
S315080049F00E461446002E02D0012E46D11CE0002D8C
S31508004A0002D0012D16D10AE0602101208007FEF7A9
S31508004A107BFF002101208007FEF7FAFF0AE06021EC
S31508004A2001208007FEF778FF002101208007FEF7A6
S31508004A30F8FF00BF00BF28E0002D02D0012D22D1CB
S31508004A4010E013480078A0420BD0602101208007AF
S31508004A50FEF75AFF214601208007FEF7D9FF0C48CA
S31508004A60047010E00B480078A0420BD060210120AA
S31508004A708007FEF751FF214601208007FEF7D1FF88
S31508004A800448047000BF00BF00BF00BF70BD00002F
S31508004A903E0100203F01002010B580211648FCF792
S31508004AA07CFF80211448FDF7AFFF0F211248FFF75E
S31508004AB0AFFC1149C98B88420AD10F482838008DA6
S31508004AC00E49884217D000F039FA00F025F812E0AE
S31508004AD00BA0FFF7ADFA00F031FA00F01DF800243C
S31508004AE007E061000448425A214608A0FFF7A0FAE9
S31508004AF0641C802CF5DB10BDBC010020FBAA00005D
S31508004B004641554C54215F310000000025642020A1
S31508004B1025640D0A2000000010B57E20FFF756FA1E
S31508004B20FDF7EAFF0848094908850F210748283094
S31508004B30FFF76EFC05492831C883802103482830D1
S31508004B40FDF780FF10BD0000FBAA000094010020BD
S31508004B5070B504460D46E1B20548FFF7ADF800BF4B
S31508004B6001210348FFF74BF80028F9D0204670BD0D
S31508004B700038014070B50446002599480088FA288F
S31508004B800ADD00209649088096490870FF21013100
S31508004B909348801DFCF701FF924800780300FFF751
S31508004BA06EFA08052031425BD5EFEDEC7E2C11D16B
S31508004BB000208B49088001208A49087088480188A6
S31508004BC00088401C864A1080901D445400201146D7
S31508004BD0C87002E0002082490880002080490871D8
S31508004BE0FBE07F4801880088401C7D4A1080901DA4
S31508004BF0445402207B490870104600790019114672
S31508004C000871EAE0764801880088401C744A1080DA
S31508004C10901D445403207349087010460079001902
S31508004C2011460871D9E06E4801880088401C6C4A14
S31508004C301080901D445404206A4908701046007973
S31508004C400019114608710846C470C078002802D1B8
S31508004C50052064490870C0E061484079012856D1AA
S31508004C605E2C1CD15E4800797E305D4908717E2134
S31508004C705B4802880088401C594B1880981D81544F
S31508004C80801FC078401EC0B21946C870002802DCD2
S31508004C9005205449087000205149487155E05D2C9B
S31508004CA01CD14F4800797D304D4908717D214C480B
S31508004CB002880088401C4A4B1880981D8154801F22
S31508004CC0C078401EC0B21946C870002802DC05200C
S31508004CD04449087000204249487136E04048007946
S31508004CE000193F490871084601880088401C3C4A5B
S31508004CF01080901D4454801FC078401EC0B21146D3
S31508004D00C870002821DC0520364908701DE07D2C76
S31508004D1003D101203249487117E03148007900195A
S31508004D202F490871084601880088401C2C4A1080C3
S31508004D30901D4454801FC078401EC0B21146C870EA
S31508004D40002802DC05202749087046E02448007937
S31508004D50C043401CC5B2A54203D1062021490870AC
S31508004D6002E007201F4908701D4801880088401C7A
S31508004D701B4A1080901D44542FE02DE01DE0FFE7EC
S31508004D80174801880088401C154A1080901D445415
S31508004D907E2C08D101211448417400201146088050
S31508004DA01049087008E000200D49088000210E48C7
S31508004DB0417400200B4908700FE00020094908706B
S31508004DC0074801880088401C054A1080901D4454F5
S31508004DD000201146088000E000BF00BF70BD00003B
S31508004DE0D80300208B010020B402002070B50246CB
S31508004DF0002013460C461D02FF2636023540254381
S31508004E00284670BD86B004460D4626686768A068C1
S31508004E100590E06804902069039060690290A06993
S31508004E200190E069009017A0FFF702F931461BA030
S31508004E30FFF7FEF839461CA0FFF7FAF81DA00599FA
S31508004E40FFF7F6F81EA00499FFF7F2F81FA00399DA
S31508004E50FFF7EEF820A00299FFF7EAF823A00199D8
S31508004E60FFF7E6F826A00099FFF7E2F82948416A15
S31508004E7029A0FFF7DDF829462BA0FFF7D9F800BFD0
S31508004E80FEE700005B48617264206661756C7420F9
S31508004E9068616E646C65725D0D0A00005230203DD3
S31508004EA02025780D0A0000005231203D2025780D76
S31508004EB00A0000005232203D2025780D0A00000025
S31508004EC05233203D2025780D0A0000005231322049
S31508004ED03D2025780D0A0000537461636B656420D4
S31508004EE04C52203D2025780D0A000000537461635A
S31508004EF06B6564205043203D2025780D0A0000008C
S31508004F00537461636B656420505352203D202578A5
S31508004F100D0A000000ED00E05343425F5348435337
S31508004F20523D25780D0A000043757272656E74202D
S31508004F304C52203D2025780D0A00000000B5154882
S31508004F4015490885FF21144841850F210186A021AE
S31508004F50C185D22181851E214186AF21C1868C213A
S31508004F600187BE2181860D49283001830B492331EB
S31508004F7041830521283841870A218187C187002175
S31508004F80283081830F21FFF743FA03492831C88364
S31508004F9000BD0000FBAA0000940100205A2500006D
S31508004FA010B55348C07D002800D110BD5048407D3B
S31508004FB0012826D14F494868C821FCF7ABFCC00731
S31508004FC0C00F002805D180210920C006FDF71DFF66
S31508004FD00DE048494868C821FCF79CFCC007C00F8B
S31508004FE0002804D080210920C006FDF710FF0821FB
S31508004FF00920C006FDF709FF01213F48FDF705FF17
S31508005000D3E73B48807C01286FD1394820300079A6
S31508005010002802D001282BD102E0FEF75DFE63E0EE
S3150800502034494868FF21F531FCF774FCC007C00F06
S3150800503000280ED180210920C006FDF7E8FE0121CF
S315080050402D48FDF7E4FE08210920C006FDF7DFFE1E
S315080050500DE080210920C006FDF7D7FE08210920AA
S31508005060C006FDF7D2FE01212348FDF7CEFE3BE040
S315080050701F4820300079052827D11E494868FF2196
S31508005080F531FCF747FCC007C00F00280ED1802178
S315080050900920C006FDF7BBFE01211748FDF7B7FE3C
S315080050A008210920C006FDF7B2FE1CE08021092070
S315080050B0C006FDF7AAFE08210920C006FDF7A5FED1
S315080050C001210D48FDF7A1FE0DE080210920C0064B
S315080050D0FDF79DFE01210848FDF799FE08210920E4
S315080050E0C006FDF794FE00BF00BF00BF5DE70000E5
S315080050F0B40200209401002000040048FEF72EFBAD
S31508005100FDF7DAFBFDF778F90B20FDF733F80920F0
S31508005110FDF730F80420FDF72DF801215348FDF777
S3150800512011FA4B200002FDF731FBFEF7B3F8FEF744
S315080051302BF8FEF749FB0D216320FEF773FB0121CF
S315080051404B48817400214175FFF7A6FCFEF7B6FCB3
S315080051507F217E20FEF75AFF86E04548007C01281D
S3150800516036D1002301221946184600F06BF90023B0
S315080051701A461946184600F065F93E4840683E4901
S31508005180884204D908213D48FDF73FFE1DE039490C
S315080051904868FF21F531FCF7BDFBC007C00F0028A2
S315080051A00ED180210920C006FDF72FFE082109200F
S315080051B0C006FDF72AFE01213048FDF726FE04E069
S315080051C008210920C006FDF722FEFDF78BFA48E004
S315080051D02748007C02283AD1FDF7DCF9FEF708F8E3
S315080051E0002301221946184600F02CF900231A4616
S315080051F01946184600F026F91E4840681E49884296
S3150800520004D908211D48FDF700FE1DE01949486824
S31508005210FF21F531FCF77EFBC007C00F00280ED131
S3150800522080210920C006FDF7F0FD08210920C006E7
S31508005230FDF7EBFD01211148FDF7E7FD04E0082124
S315080052400920C006FDF7E3FDFFF732FB09E0FDF78D
S31508005250A1F9FFF7A5FEFFF7EFF8FDF7C9FF00F084
S3150800526037FA7E20FEF7B2FE77E7000000240140F9
S31508005270B402002094010020204E000000040048DB
S31508005280F7B5A0B00C46154680216846FCF785FBA5
S31508005290002700267E2168460170FE214170EF2115
S315080052A081700721C17020990171002141718471B3
S315080052B02112C171012101724572291281720126DA
S315080052C005E06846805DC019C7B2701CC6B20B2ED1
S315080052D0F7DBF843401CC1B26846C1727E210173F0
S315080052E00D21FEF757FC23B0F0BDFFB585B0054686
S315080052F00E460E9F002001900290039004900090A5
S3150800530000247E2168460171457186710421C171A8
S31508005310079901720899417287723912C17201247C
S3150800532007E001A8015D00980818C0B20090601C4B
S31508005330C4B2082CF5DB0098C043401CC1B26846CD
S3150800534001737E2141730A2101A8FEF723FC09B0E7
S31508005350F0BDF7B584B005460E46002000900190D2
S3150800536002900390002700247E216846017046704B
S3150800537085700121C170694606980871012405E007
S315080053806846005DC019C7B2601CC4B2052CF7DBBD
S31508005390F843401CC1B2684641717E2181710721DC
S315080053A0FEF7F8FB07B0F0BD70B504460D467E2043
S315080053B0FEF70CFE03E02078641CFEF7DBFB2846AC
S315080053C0691E8DB20028F6D170BD000030B5A1B0B7
S315080053D00446802101A8FCF7E0FA0025002C02D03B
S315080053E0012C20D10FE07E21684601710021417110
S315080053F0442181711321C1711522104902A8FCF7B5
S31508005400B3FA192510E07E2168460171FE21417123
S31508005410442181713321C1713622094902A8FCF75A
S31508005420A3FA3A2500E000BF00BF802D03DA29461B
S3150800543001A8FFF7B9FF21B030BD000040010020E8
S3150800544055010020FFB583B006460C4617460020D6
S31508005450029000259A480078642803D09948007875
S31508005460642803D101219848817502E000219648F5
S315080054708175002F02D0012F64D164E09348C08E55
S31508005480A04202D19148C58F00E00525052D01DC13
S31508005490052502E0322D00DB0525601BB0420BDD39
S315080054A08948C07E00280DD18848406887498861A8
S315080054B001218548C17605E06019B04202DC002169
S315080054C08148C1768048C07E012832D17C48007860
S315080054D07C490978884203DA0020794908702BE06C
S315080054E0601BB0421ADD7948808E642806DB64208A
S315080054F0734908700121744881751DE07349888EC7
S31508005500C10F091849103C316D4A117010460078D0
S31508005510642811DD6420114608700DE01E2D03DD98
S3150800552064206749087007E02846463064490870D1
S3150800553002E00020624908706148027838460699F8
S31508005540FFF754FAB7E0604820300079022808D1FE
S315080055505E48408DA04202D15C48458F17E00A2577
S3150800556015E0594820300079032808D15748808D1E
S31508005570A04202D15548858F09E00A2507E053481D
S31508005580808DA04202D15148858F00E00A25052D5D
S3150800559001DC052502E0322D00DB3225601BB04216
S315080055A00BDD4948007F002815D14848406847491F
S315080055B0C8610121444801770DE06019B0420ADC50
S315080055C04148007F012806D1404840683F49C861E4
S315080055D000213D4801773C48007F01283CD13948E5
S315080055E0007837490978884203DA00203549087077
S315080055F05AE0601BB0420ADD50203249087001218A
S3150800560031488175314840683049C8614CE0052108
S315080056102846FCF795F92D4949682C4AD269891A12
S3150800562048437D21C9000190FCF774F90019B0427E
S315080056300ED950202349087023482038808DB22877
S3150800564032DA0121214828308183FFF765FA2BE0F9
S3150800565000201C49087027E01C4949681B4AD26982
S31508005660881A7D21C900FCF755F9082819D805219B
S315080056702846FCF765F915494968144AD269891A12
S3150800568048437D21C9000190FCF744F9201AB0422D
S3150800569003D350200B49087006E00020094908701A
S315080056A002E000200749087006480278384606993D
S315080056B0FFF79CF900BF00BF029807B0F0BD0000D5
S315080056C0C2000020C3000020B4020020940100207C
S315080056D010B5F748007900285BD00020F549088006
S315080056E0F3484038408DFF217D31884204DCF0487C
S315080056F04038008D88420ADDED482038407D002874
S3150800570005D1ED4948600121E94820384175EA4844
S31508005710006AEA4988420AD9E5482038407D0028C7
S3150800572005D1E54948600121E14820384175E0483E
S315080057302038407D01282CD1DD482038807C01287E
S3150800574027D10023012219461846FFF77BFE0023BE
S315080057501A4619461846FFF775FED74840687D2150
S315080057600901884214D90020D34948600821092034
S31508005770C006FDF74AFB80210920C006FDF745FB58
S315080057800121CF48FDF741FB0021C9482038817423
S3150800579010BDC7482038807C002848D10821092038
S315080057A0C006FDF732FB80210920C006FDF72DFB58
S315080057B00121C348FDF729FB002301221946184693
S315080057C0FFF740FE00231A4619461846FFF73AFE29
S315080057D0B9484068FF21F531884204D20421B84807
S315080057E0FDF715FB42E27D20C000B349486004215D
S315080057F0B348FDF70AFBAE482038807E002809D159
S315080058000821AF48FDF701FB0021A948203841755A
S3150800581041762BE24021AA48FDF7EEFA0028E1D0AE
S315080058200021A34801710121203881741EE2A04895
S3150800583000790300FEF723FC06044AD7FEFDFC495F
S315080058400023012219461846FFF7FCFD00231A46D5
S3150800585019461846FFF7F6FD95482038007C0128BA
S3150800586009D1954800699749884203D9002190488B
S31508005870203801748CE7904840687D2109018842E8
S315080058801FD900208C49486040218D48FDF7B4FA9D
S31508005890002807D108218A48FDF7B7FAFF20F53016
S315080058A0FCF7CCFF08210920C006FDF7AEFA8021D7
S315080058B00920C006FDF7A9FA01218148FDF7A5FAD6
S315080058C003E008217E48FDF7A2FACEE17A4840684F
S315080058D0FF21F531884204D204217948FDF797FA69
S315080058E003E004217648FDF790FA734948687D215C
S315080058F0C900FCF70FF823281CD26F4948687D2198
S31508005900C900FCF707F8192814D969484038018DE9
S315080059106948408D814206DA65484038418D6648B7
S31508005920408D814214DB00206349486002216048AB
S3150800593001710DE0604948687D21C900FBF7EAFF5F
S31508005940232805D300205C49486002215848017184
S3150800595057484038408DFF217D31884204DC544841
S315080059604038008D88420CDD00230122194618466E
S31508005970FFF768FD00231A4619461846FFF762FD29
S3150800598030E04D48418D408F091849484038408DD0
S31508005990814210DD642201210846FFF727F801211C
S315080059A0434820388175407E002815D1002140489B
S315080059B02038417610E04048418D408F09183C4810
S315080059C04038408D814207DC01213948203841762C
S315080059D000220846FFF70AF800231A461946184611
S315080059E0FFF730FD41E134484068FF21F531884230
S315080059F004D204213248FDF70AFA03E004213048AC
S31508005A00FDF703FA2A484038408DFF217D31884248
S31508005A1004DC27484038008D884210DD0023012227
S31508005A2019461846FFF70EFD00231A46194602E0E6
S31508005A30A9E06AE022E01846FFF704FD1DE01E48CB
S31508005A404168008E7D22D200504381420FD21A4A05
S31508005A50518DFF320132508D01231A46FFF7F2FCB1
S31508005A6000231A4619461846FFF7ECFC05E0002005
S31508005A701149486003210E480171F6E00C48403888
S31508005A80408DFF217D31884204DC09484038008D6D
S31508005A90884219DD0023012219461846FFF7D2FC71
S31508005AA000231A4619461846FFF7CCFC2CE00000DE
S31508005AB0D4020020C40000209401002070110100C7
S31508005AC00004004888130000694948687D21C90018
S31508005AD0FBF720FF6649498E88420FD2644A918DAA
S31508005AE0FF320132508D01231A46FFF7ABFC002323
S31508005AF01A4619461846FFF7A5FC05E000205C493A
S31508005B00486004215B480171AFE05A484038408D2F
S31508005B10FF217D31884204DC56484038008D884292
S31508005B200CDD0023012219461846FFF78BFC0023DB
S31508005B301A4619461846FFF785FC23E04C4948687B
S31508005B407D21C900FBF7E6FE4949098F0F398842CE
S31508005B5012D2474AD18EFF320132108D012300221C
S31508005B60FFF770FC424AD18DFF320132508D012376
S31508005B701A46FFF767FC05E000203D494860052105
S31508005B803C48017171E03A484068FF21F531884286
S31508005B9004D204213848FDF73AF90FE03448406842
S31508005BA0FF21F531884209D9314840684B21C9009F
S31508005BB0884203D204213048FDF727F92C4840686B
S31508005BC02E4988422BD22B484038408DFF21193167
S31508005BD0884204DC27484038008D88420CDD0023C3
S31508005BE0012219461846FFF72DFC00231A461946C6
S31508005BF01846FFF727FC37E01D4AD18EFF320132DF
S31508005C00108D01230022FFF71DFC194AD18DFF32A2
S31508005C100132508D01231A46FFF714FC24E00421B3
S31508005C201548FDF7F4F812484068154988421BD311
S31508005C3000201449088000210E480171203881741B
S31508005C400023012219461846FFF7FCFB00231A46D3
S31508005C5019461846FFF7F6FB04210748FDF7D5F85D
S31508005C6008210548FDF7D1F800BF00BF00BF8FE542
S31508005C7094010020D402002000040048A438000043
S31508005C80983A0000C4000020A85C0008C000002064
S31508005C90D4000000144100087C5D0008940100202F
S31508005CA04C07000024410008000000000000000026
S31508005CB000000000010203040102030406070809A4
S31508005CC000A24A04000000000000000001020304CC
S31508005CD00607080900000000000000000000000098
S31508005CE000000000040000000100000000000000A1
S31508005CF00000000000000000000000000000000096
S31508005D000000000000000000000000000000000085
S31508005D100000000000000000000000000000000075
S31508005D20000000000000000000011058594C4C30DB
S31508005D303131327878787878787878CB7E000110A7
S31508005D4058594C4C30313132787878787878787878
S31508005D5004013205054C4C303131061459413230B4
S31508005D603035323848343530343241787878787876
S31108005D707D5D7E000000000000000000C1
S705080018C515
